:10000000B4016E2A8C21B6000408B80008008C21C7
:10001000B7000408B90008000408A200831686117E
:1000200083120930A30003101C20A20CA30B142878
:1000300003141C200314692A0318212800008615C4
:100040002328861123280030A100C330D7290408B3
:10005000A7000610861086108316061086108610DC
:100060000F30860583122708B41854283A30A100AF
:100070009830D7213330A60068201330A100883093
:10008000D72168206430D62168206430D621223000
:10009000A6006820283053200C305320063053200F
:1000A000B414270854283414A600341C622886107F
:1000B000033C031C672867200730A100D030D721FC
:1000C000031408003414FE3C0319692A8614341CF6
:1000D000341006140F3086052608F0398604061001
:1000E000A60E341868283230D621031408008C215B
:1000F000B6008821200821040319692A5E2284138E
:1001000036088006640084288528A00A0319A10FF8
:1001100082288006692A6400A12003188B28E82021
:10012000A8010830A300E920A1200318A80AAB1EEB
:10013000A801A20CA30B9328AB1AA213E920220852
:1001400008003808840036088417800484130005EA
:100150002B1B3606FF3E0800A401A501B512642240
:10016000D33E0319B5162D3EC63E0318BB280A3EE2
:10017000031CAF28C228F33E0318AF28063E031C19
:10018000AF280A3EA2000430A3000310A40DA50D61
:10019000A30BC5282208A404A9030319DF2864229D
:1001A000C63E0318D7280A3E031CDF28C228F33EA8
:1001B0000318DF28063E031CDF280A3EC228B51EAE
:1001C000E628A409A509A40A0319A50A2408692A8E
:1001D00035172B081F39FF3EA1002A08F53E0318EA
:1001E000A10A351FD7293513A00002300922D729CB
:1001F000B51329080319B5170430A800250E0521E9
:1002000025080521240E052124080F39F63E031880
:10021000073E0A3E2829B51329080319B5170530EA
:10022000A8002730A300103021210330A300E830BC
:100230002121A30164302121A3010A3021212408B6
:100240002829A2002508A1002408A0002C222008AB
:10025000A000A8030319B51329080319322928029D
:10026000031808002008031DB513B51B0800303E15
:10027000642A0830A600A700390884003708351919
:100280008004FF3A351D800589213808840036082E
:100290008521A001A101B518792138088400000842
:1002A0003605FF3EA00DA10DB51C7921A60B4B29EB
:1002B00027083518EB292008692A0830A6003518C8
:1002C000EB2139088400370835198021351D82213A
:1002D000380884003609892138088400A10CA00C54
:1002E00000083604031C360680007921A60B6C2911
:1002F000692A390884003708800600008006080053
:1003000080048829FF3A8005892984178004692A96
:10031000FF3A84178005692AA8000630A81907301B
:10032000840001308A00280807398207013402342A
:10033000043408341034203440348034A000A00D3C
:10034000A00DA00D3830A005813020049F000030A2
:10035000A1003230D7211F151F19AC291E08A1009A
:1003600083161E08692A03178D0083168C130C143C
:1003700083120C08692A03178C0083168C130C1542
:1003800055308D00AA308D008C148C18C5290C11A5
:10039000692AA301A200FF30A207031CA307031CC4
:1003A000692A0330A100DF30D721CB29A101E83E23
:1003B000A000A109FC30031CE029A0070318DD29D7
:1003C000A0076400A10FDD292018E629A01CEA2956
:1003D0000000EA290800A400A201A301F329A10C4E
:1003E000A00CA20DA30DFF3E0318EF292408012243
:1003F0002208A0042308A104200808000310A00D6F
:10040000A10DFF3E0318FE292008692A0310A10C44
:10041000A00CFF3E0318062A2008692AA200033018
:100420001C2AA20001301C2AA20006301C2AA200AD
:1004300004301C2AA2000530A80023082102031D55
:10044000232A220820020430031801300319023045
:100450002805031DFF30692A1030A600A501A4015C
:10046000210DA40DA50D2208A4022308031C230FAF
:10047000A5020318422A2208A40723080318230F01
:10048000A5070310A00DA10DA60B302A2008692A8C
:100490001030A800A101A001A70CA60C031C562A2D
:1004A0002208A00723080318230FA107A10CA00C02
:1004B000A50CA40CA80B4C2A2408692AA009A109A0
:1004C000A00A0319A10A0800840031088A00300834
:1004D0008200831303138312640008000330A30017
:1004E000E8308A01CA218316043086003F30850037
:1004F000FC3087008312831684309F008312813082
:100500009F006430F900F8016430F200F1011F30FF
:10051000C2000430C3002030C0000330C1000130ED
:10052000BC00BD010130EE0064008A110A12071EF2
:10053000A02A64008A110A12071A5D2F8A01942AE0
:10054000FE308A01282001308A01282043308A01A8
:10055000282061308A0128206C308A0128206930E7
:100560008A01282062308A01282072308A012820DE
:1005700061308A01282063308A01282069308A018D
:1005800028206F308A0128206E308A0128204330CD
:100590008A010D2061308A010D206C308A010D2006
:1005A00069308A010D2062308A010D2072308A0183
:1005B0000D2061308A010D2063308A010D206930E1
:1005C0008A010D206F308A010D206E308A010D20C6
:1005D00020308A010D202D308A010D2020308A0123
:1005E0000D2065308A010D206E308A010D20743097
:1005F0008A010D2072308A010D2061308A010D20A0
:1006000072308A010D2020308A010D2076308A0157
:100610000D2061308A010D206C308A010D206F3071
:100620008A010D2072308A010D2065308A010D206B
:1006300073308A010D200A308A010D200D308A01A5
:100640000D2043308A010D206F308A010D206D305E
:100650008A010D2070308A010D2065308A010D203D
:100660006E308A010D2073308A010D2061308A01BD
:100670000D2063308A010D2069308A010D206F3012
:100680008A010D206E308A010D2020308A010D2054
:1006900054308A010D2065308A010D206D308A01A9
:1006A0000D2070308A010D202B308A010D203A3048
:1006B0008A010D200A308A010D200D308A010D209B
:1006C0000530B8002030B600BC30AA004030AB0086
:1006D0000130A9008B30B000B1018A01AC20F400D8
:1006E0000130A9007408A400A5010C30B000B101CC
:1006F0008A01F8200A308A010D200D308A010D2070
:10070000FE308A012820C0308A01282054308A0116
:10071000282065308A0128206D308A012820703019
:100720008A01282020308A0128202B308A012820A5
:100730000130A9007408A400A5012730B000B10160
:100740008A01F820031701308D00031374088A0111
:10075000BB210330A300E8308A01CA21FE308A01A0
:10076000282001308A01282043308A012820613066
:100770008A0128206C308A01282069308A012820CB
:1007800062308A01282072308A01282061308A0173
:10079000282063308A01282069308A0128206F30A0
:1007A0008A0128206E308A01282043308A010D20DA
:1007B0006F308A010D206D308A010D2070308A0162
:1007C0000D2065308A010D206E308A010D207330B6
:1007D0008A010D2061308A010D2063308A010D20CD
:1007E00069308A010D206F308A010D206E308A0138
:1007F0000D2020308A010D2054308A010D206530F3
:100800008A010D206D308A010D2070308A010D2083
:100810002D308A010D203A308A010D200A308A01DC
:100820000D200D308A010D200530B8002030B600B3
:10083000BC30AA004030AB000130A9008B30B000C2
:10084000B1018A01AC20F4000130A9007408A400B1
:10085000A5010C30B000B1018A01F8200A308A01EC
:100860000D200D308A010D20FE308A012820C03075
:100870008A01282054308A01282065308A012820E6
:100880006D308A01282070308A01282020308A01AA
:1008900028202D308A0128200130A9007408A400E6
:1008A000A5012730B000B1018A01F82003170230FA
:1008B0008D00031374088A01BB210330A300E830C4
:1008C0008A01CA21FE308A01282001308A012820AD
:1008D00043308A01282061308A0128206C308A0147
:1008E000282069308A01282062308A01282072304D
:1008F0008A01282061308A01282063308A0128205B
:1009000069308A0128206F308A0128206E308A01E0
:10091000282043308A010D206F308A010D206D3070
:100920008A010D2070308A010D2065308A010D206A
:100930006E308A010D2073308A010D2061308A01EA
:100940000D2063308A010D2069308A010D206F303F
:100950008A010D206E308A010D2020308A010D2081
:1009600048308A010D2075308A010D206D308A01D2
:100970000D202B308A010D203A308A010D200A30DB
:100980008A010D200D308A010D200530B80020307D
:10099000B600BC30AA004030AB000130A9008B305B
:1009A000B000B1018A01AC20F4000130A900740844
:1009B000A400A5010C30B000B1018A01F8200A3072
:1009C0008A010D200D308A010D20FE308A01282079
:1009D000C0308A01282048308A01282075308A01D9
:1009E00028206D308A01282020308A0128202B30D1
:1009F0008A0128200130A9007408A400A50127302D
:100A0000B000B1018A01F820031703308D000313F1
:100A100074088A01BB210330A300E8308A01CA218F
:100A2000FE308A01282001308A01282043308A01C3
:100A3000282061308A0128206C308A012820693002
:100A40008A01282062308A01282072308A012820F9
:100A500061308A01282063308A01282069308A01A8
:100A600028206F308A0128206E308A0128204330E8
:100A70008A010D206F308A010D206D308A010D2012
:100A800070308A010D2065308A010D206E308A0198
:100A90000D2073308A010D2061308A010D206330F2
:100AA0008A010D2069308A010D206F308A010D20E6
:100AB0006E308A010D2020308A010D2048308A01D5
:100AC0000D2075308A010D206D308A010D202D30EA
:100AD0008A010D203A308A010D200A308A010D204A
:100AE0000D308A010D200530B8002030B600BC3032
:100AF000AA004030AB000130A9008B30B000B1013A
:100B00008A01AC20F4000130A9007408A400A501FA
:100B10000C30B000B1018A01F8200A308A010D20A2
:100B20000D308A010D20FE308A012820C0308A0154
:100B3000282048308A01282075308A0128206D300D
:100B40008A01282020308A0128202D308A0128207F
:100B50000130A9007408A400A5012730B000B1013C
:100B60008A01F820031704308D00031374088A01EA
:100B7000BB210330A300E8308A01CA21FE308A017C
:100B8000282001308A01282043308A012820613042
:100B90008A0128206C308A01282069308A012820A7
:100BA00062308A01282072308A01282061308A014F
:100BB000282063308A01282069308A0128206F307C
:100BC0008A0128206E308A01282043308A010D20B6
:100BD0006F308A010D206D308A010D2070308A013E
:100BE0000D2065308A010D206E308A010D20733092
:100BF0008A010D2061308A010D2063308A010D20A9
:100C000069308A010D206F308A010D206E308A0113
:100C10000D2020308A010D2050308A010D207230C5
:100C20008A010D2065308A010D2073308A010D2064
:100C300073308A010D202B308A010D203A308A0151
:100C40000D200A308A010D200D308A010D2005305B
:100C5000B8002030B600BC30AA004030AB000130F4
:100C6000A9008B30B000B1018A01AC20F400013042
:100C7000A9007408A400A5010C30B000B1018A01DC
:100C8000F8200A308A010D200D308A010D20FE3037
:100C90008A012820C0308A01282050308A0128206B
:100CA00072308A01282065308A01282073308A0139
:100CB000282073308A01282020308A0128202B30F8
:100CC0008A0128200130A9007408A400A50127305A
:100CD000B000B1018A01F820031705308D0003131D
:100CE00074088A01BB210330A300E8308A01CA21BD
:100CF000FE308A01282001308A01282043308A01F1
:100D0000282061308A0128206C308A01282069302F
:100D10008A01282062308A01282072308A01282026
:100D200061308A01282063308A01282069308A01D5
:100D300028206F308A0128206E308A012820433015
:100D40008A010D206F308A010D206D308A010D203F
:100D500070308A010D2065308A010D206E308A01C5
:100D60000D2073308A010D2061308A010D2063301F
:100D70008A010D2069308A010D206F308A010D2013
:100D80006E308A010D2020308A010D2050308A01FA
:100D90000D2072308A010D2065308A010D207330DC
:100DA0008A010D2073308A010D202D308A010D201B
:100DB0003A308A010D200A308A010D200D308A0157
:100DC0000D200530B8002030B600BC30AA004030FD
:100DD000AB000130A9008B30B000B1018A01AC201A
:100DE000F4000130A9007408A400A5010C30B00083
:100DF000B1018A01F8200A308A010D200D308A01E4
:100E00000D20FE308A012820C0308A012820503071
:100E10008A01282072308A01282065308A01282022
:100E200073308A01282073308A01282020308A01FB
:100E300028202D308A0128200130A9007408A40040
:100E4000A5012730B000B1018A01F8200317063050
:100E50008D00031374088A01BB210330A300E8301E
:100E60008A01CA21FE308A01282001308A01282007
:100E700050308A01282075308A0128206C308A0180
:100E8000282073308A01282061308A01282072309E
:100E90008A01282020308A01282052308A01282007
:100EA00065308A01282073308A01282065308A0144
:100EB000282074308A0128200800FE308A0128206A
:100EC00001308A01282057308A01282045308A01C4
:100ED000282041308A01282054308A0128204830B7
:100EE0008A01282045308A01282052308A01282092
:100EF00020308A01282020308A01282053308A019E
:100F0000282054308A01282041308A01282054307A
:100F10008A01282049308A0128204F308A01282060
:100F20004E308A012820FE308A012820C0308A01F4
:100F3000282020308A01282045308A01282041308D
:100F40008A01282033308A01282043308A01282052
:100F50004E308A0128204F308A01282020308A0113
:100F6000282020308A01282050308A01282049304A
:100F70008A01282043308A0128205F308A012820F6
:100F800057308A01282058308A01282020308A01D1
:100F900028200B30A300B8308A01CA218716831697
:100FA00087120F3083128A0102200E308A01072037
:100FB000B5010C30A000A1018A015D210230A00022
:100FC000A1018A015D2187128316871283120030E6
:100FD0008A019E21E60001308A019E21BA00210883
:100FE000BB0003308A019E21E7000330A300E830F4
:100FF0008A01CA2101308A01B321ED0002308A0141
:10100000B321EC0003308A01B321E90004308A01E6
:10101000B321E80005308A01B321EB0006308A01D4
:10102000B321EA008A150A12BA218A150A12F82198
:101030008A150A1210228A150A1284228A150A12A7
:10104000A2223E08A0003F08A1004508A3004408D2
:101050008A0114228A150A12031D30287E30EF00FF
:101060003E08A0003F08A1004508A30044088A01EB
:101070001A228A150A12031D3F283D30EF003E0850
:10108000A0003F08A1004508A30044088A010E22E1
:101090008A150A12031D4E287F30EF00FE308A01A8
:1010A000282001308A01282020308A0128202B3076
:1010B0008A0128200230A9007508A400A501273064
:1010C000B000B1018A010B212E308A0128200130A5
:1010D000A9007708A400A5012730B000B1018A015A
:1010E0000B21DF308A01282043308A01282020305C
:1010F0008A01282020308A0128200230A9007008A7
:10110000A400A5012730B000B1018A010B212530D0
:101110008A01282052308A01282048308A0128205C
:1011200020308A012820FE308A012820C0308A0120
:10113000282020308A01282020308A0128202030D1
:101140008A0128200430A9003E08A4003F08A50019
:101150002730B000B1018A010B2120308A012820FC
:1011600068308A01282050308A01282061308A01A5
:10117000282020308A0128206F088A01282020306A
:101180008A01282020308A01282020308A01282046
:101190000A308A01C92164008A150A12871D012BB1
:1011A00064008A150A12071E822B8A150A12B222BF
:1011B0008A150A12C7228A150A12DC22BC0A0319F0
:1011C000BD0A3C08A0003D08A1000130A300213069
:1011D0008A0114228A110A12031DE72F2E308A0178
:1011E0000D202E308A010D202E308A010D202C304A
:1011F0008A010D202E308A010D202E308A010D200B
:101200002E308A010D202C308A010D202E308A01CB
:101210000D202E308A010D202E308A010D202C3019
:101220008A010D200330A9004A08A4004B08A5003C
:101230000C30B000B1018A010B212C308A010D2045
:101240000430A9003E08A4003F08A5000C30B000FF
:10125000B1018A010B212C308A010D200230A90036
:101260007008A400A5010C30B000B1018A010B2167
:101270002C308A010D202E308A010D202E308A015B
:101280000D202E308A010D202C308A010D202E30A9
:101290008A010D202E308A010D202E308A010D206A
:1012A0002C308A010D202E308A010D202E308A012B
:1012B0000D202E308A010D202A308A010D202E307B
:1012C0008A010D202E308A010D202E308A010D203A
:1012D0002C308A010D202E308A010D202E308A01FB
:1012E0000D202E308A010D202C308A010D202E3049
:1012F0008A010D202E308A010D202E308A010D200A
:101300002A308A010D202A308A010D200230A900DE
:101310007508A400A5010C30B000B1018A010B21B1
:101320002E308A010D20A9017708A400A5010C30F8
:10133000B000B1018A010B210A308A010D200D3065
:101340008A010D200130BC00BD01EE0A64000B30A3
:101350006E028A110A12031CE72F3E08C4003F08E0
:10136000C5000130EE000330A300E8308A01CA2135
:101370008A01E72F8716831687120F3083128A019E
:1013800002200E308A010720B501EE30A000A10135
:101390008A015D21871283168712831287168316AE
:1013A00087120F3083128A0102200E308A01072033
:1013B000B501AA30A000A1018A015D210F308A0188
:1013C00002200E308A0107200130B5008A01392140
:1013D000CA002108CB0087128316871283126D087A
:1013E000CA070318CB0A6C08CA02031CCB03080007
:1013F0004B0C4A0CF5004A08A0004B08A100023033
:10140000A200A3018A012C222408F6007608A60077
:10141000A7010530A200A3018A014822F7000800B5
:101420003A08A6003B08A7003230A200A3018A01B7
:101430004822B2002508B3003208A0003308A100FA
:10144000FF30A2000330A3008A012C22C60021082D
:10145000C7003A08A6003B08A7003230A200A3014B
:101460008A014822B2002508B3003208A0003308E0
:10147000A100FF30A2000330A3008A012C2224081F
:10148000C8002508C9004608A6004708A700E8309C
:10149000A2000330A3008A014822B2002508B3004D
:1014A0004808B20749080318013EB3073208A000F4
:1014B0003308A100F430A2000130A3008A012C22DD
:1014C000B2002108B3001030B2020030031C013E0C
:1014D000B3023208A6003308A7006430A200A301BB
:1014E0008A014822B2002508B3003208A000330860
:1014F000A1003E30A200A3018A012C22F00069085D
:10150000F0076808F002080007108316071083121E
:1015100087108316871083126430A000A101093060
:101520008A0177200A308A01022009308A010720C7
:101530000230B5008A013921F30007148316071021
:101540008312080020307307BE0003300318013EE9
:10155000BF006B08BE070318BF0A6A08BE02031C5F
:10156000BF0308006400750878028A150A12031C7C
:10157000C12A6400790875028A150A12031CC42A5C
:1015800008007508F80008007508F90008006400F4
:10159000700871028A150A12031CD62A64007208A8
:1015A00070028A150A12031CD92A08007008F1007B
:1015B00008007008F20008003E08A0003F08A100E3
:1015C0004108A30040088A0111228A150A12031D4E
:1015D000F72A3E08A0003F08A1004308A3004208E4
:1015E0008A0117228A150A12031DFC2A08003E08E8
:1015F000C0003F08C10008003E08C2003F08C30009
:101600000800FE308A01282001308A012820DF30BE
:101610008A01282043308A01282020308A0128208E
:1016200020308A01282020308A0128204D308A016C
:10163000282020308A0128202B308A0128200230DF
:10164000A9007808A400A5012730B000B1018A01E3
:101650000B2120308A0128206D308A01282020307B
:101660008A0128202B308A0128200230A90079081D
:10167000A400A5012730B000B1018A010B21FE3082
:101680008A012820C0308A01282025308A0128209C
:1016900052308A01282048308A01282020308A01CF
:1016A000282020308A0128204D308A01282020302F
:1016B0008A01282020308A0128200230A9007108E0
:1016C000A400A5012730B000B1018A010B21203010
:1016D0008A0128206D308A01282020308A012820A4
:1016E00020308A0128200230A9007208A400A50138
:1016F0002730B000B1018A010B2164308A01C92171
:101700008A01E72FFE308A01282001308A01282033
:1017100068308A01282050308A01282061308A01EF
:10172000282020308A0128204D308A0128200430CA
:10173000A9004008A4004108A5002730B000B1016D
:101740008A010B2120308A0128206D308A0128204F
:101750000430A9004208A4004308A5002730B000C7
:10176000B1018A010B2120308A012820FE308A0134
:101770002820C0308A01282064308A01C9218A01CA
:02178000E72F51
:02400E00753DFE
:00000001FF
